:030000000219FDE5
:03000B000200AA46
:03002B0002015C73
:03005B000202E8B6
:030073000202D5B1
:1000800002030406080C10182030406080040608A3
:100090000C10182030406080A0C00003070F1F0D17
:1000A0000D0403060D0503030202C2AFC0D0C0E079
:1000B000206214E5256009E473E525F4F58AD2622F
:1000C000D0E0D0D0D2AF3285268AC262E526F46075
:1000D0002F30682520720DD0E0D0D0C292C290C2DD
:1000E00091D2AF32C292C290C291206F0C206509AA
:1000F000740AD5E0FDE57B4290D0E0D0D0D2AF329B
:10010000758A00C28DD26201F901B9306805206597
:1001100002D29201B9306805206502D29101B9304E
:100120006805206502D29001B9C29530680A206541
:10013000077408D5E0FDD29201B9C29430680A2054
:1001400065077408D5E0FDD29101B9C29330680A01
:100150002065077408D5E0FDD29001B9C2AFC2ADE9
:1001600053E6EFC0D0C0E0D2D3D2AFC2CEE52A6012
:1001700007207449152A21BD7800790020742EE5E6
:1001800080307E01F430E70278FF53DACF207E031F
:1001900043DA20307E0343DA10C2D8C271E58030E2
:1001A0007E01F430E70279FFC3E89970CB30610338
:1001B000752A40207403752A40885CD27020740D23
:1001C000E52B6004152B21CD43DA01C2D820700243
:1001D00021E0A85C206102C27020740221DE882226
:1001E0007882B6040385222420CF0AD0E0D0D04301
:1001F000E610D2AD32C2CF053A7802E52A6005306A
:100200007402152AC3E55C94014005755F00412125
:10021000756000756900E55F2401F55F5003755F47
:10022000FF7982B7020D306E1DC3E522943240166D
:10023000854C227982B7030E306E0BC3E5229432CF
:100240004004798E8722C3E5239522600840041577
:100250002341550523D8CA0569E56970021569D59A
:100260006A69756A017808E56B60497805C3E569D4
:10027000956B4057C3E569956C50087801756A0322
:1002800002028FC3E569956D50057801756A01C357
:10029000E5629524401E7982B7040241C0206E14A5
:1002A000852462E569046003856B69756A017523BD
:1002B0003C0202CBE5622850057562FF41C0F56241
:1002C000E5620470067560FF7569FFD0E0D0D04329
:1002D000E610D2AD32C2AF53E67F7592FA7593FF46
:1002E000C260759104D2AF32C2AF53E6EFC2ADC067
:1002F000D0C0E0C0F0D2D3D2AFA8FBA9FCC2D830A6
:100300007102614F53DACF207E0343DA10307E034F
:1003100043DA20D271E580307E01F420E7026126C5
:1003200088278928A13453DACF207E0343DA20308E
:100330007E0343DA10C2D8C271307402A120780063
:10034000E580307E01F430E702A120885CA10853EB
:10035000DACF207E0343DA20307E0343DA10C27105
:10036000206102812853DACF207E0343DA10307EE9
:100370000343DA20C2D8D27188578958C3E895550B
:10038000F8E99556F97B007E087A00C3E8948CE979
:1003900094005005755B00811A882178A2E6A82197
:1003A0006055C3E894C8E994005008E4D2E4FB7AAD
:1003B0000A61F5C3E89468E994015008E4D2E3FBCC
:1003C0007A0F61F5C3E894D0E994025008E4D2E2D0
:1003D000FB7A1E61F5C3E894A0E994055008E4D2C5
:1003E000E1FB7A3C61F5C3E89498E994085008E48D
:1003F000D2E0FB7A787E00C3E89559FCE9955AFD76
:1004000030E70AECF42401FCEDF43400FD755B00E8
:10041000C3EC9AED9E5003755B018859895A855744
:10042000558558567802A108C3E89527F8E995281C
:10043000F9307C0281EC307B0281EC307A0281E57C
:10044000207502814BE9FDE8FC816AE9C313F9E8F4
:1004500013F830790281E5E9C313F9E813F830782D
:100460000281E5E9C313FDE813FC20612CC3EC9481
:0F0470001CED940240028181ED701EC3EC94C814
:10047F0050180529E52970021529C3E529940A505A
:10048F0002A120755C00D270A120E5296002152918
:10049F007400207F037896E624FAFEE43400FFC34D
:1004AF00EC9EFCED9FFD50067800790081ECC3ECCB
:1004BF0094FFED9400400678FF790081ECEC857293
:1004CF00F0A4C5F0A2F733F87900400302050878CD
:1004DF00FF7900020508E9C313F9E813F8307C0E21
:1004EF00E9600278FFC3E81338F8E43400F9C3E891
:1004FF0094FFE99400400278FF885CD2702061027B
:10050F00A120741FF4552F4BF52FC274EB7002D23C
:10051F0074752A40307403752A0A306102A13420A1
:10052F00740353DAFE207403752B20D0F0D0E0D083
:10053F00D0D2AD43E610327901020564790302058A
:10054F0064790A020564791E020564796402056400
:10055F0079C80205647817E4D5E0FDD8FAD9F622F8
:10056F007A147B7802058B7A107B8C02058B7A0DBF
:10057F007BB402058B7A0B7BC802058BE573D5E044
:10058F0001227902E4C294D5E0FDD291D5E0FDC2FB
:10059F0091D5E0FDD294D5E0FDE920E002D2923072
:1005AF00E002D290E573D5E0FDE920E002C292307F
:1005BF00E002C2907496D5E0FDD9C9EAF8D5E0FD06
:1005CF00D8FBDBB8C29422C37C007D0075F0000518
:1005DF00F0EA33FAEB33FB50F6EB13FBEA13FAC3F3
:1005EF00E9FFE8FEE89AF8E99BF95004EFF9EEF815
:1005FF00B3EC33FCED33FDD5F0DFEDF9ECF822E889
:10060F0089F08A20D2D4F8A9F07B0030F70B7BFF5A
:10061F00F42401F8E9F43400F9E88520F0A4ADF0F2
:10062F00F8E98520F0A4AFF0FEED2EF974003FFA43
:10063F007C04C3EA13FAE913F9E813F8DCF48BF03E
:10064F0030F70AE8F42401F8E9F43400F9E889F006
:10065F00C2D4F8A9F0227882B60403020704C3E5D6
:10066F005C9419401EE52D54067018206E367805DF
:10067F007994E7146007780A1460027812C3E54191
:10068F0098401F306E098564627569FF756A018530
:10069F002224E4F544F545F546F547F548C26E02C8
:1006AF000704D26E7994E7147013E523F43333F90A
:1006BF0013F8E9540104F9E854FE0206F8E714149C
:1006CF007014E523F4333333F913F8E9540304F9C1
:1006DF00E854FC020700E523F433333333F913F8FE
:1006EF00E954070404F9E854F8C39440F8E9940076
:1006FF00F98844894522C3E54113F9E54013F8C34E
:10070F00E54498F8E54599F9500CC3E89480E994CD
:10071F00FF401602073CC3E8947FE99400500302A0
:10072F00073C787F790002073C788079FF884989F8
:10073F004A22E5492546F8E54A3547F9854A20E436
:10074F00300701F43548FA30E709C3EA94F0401551
:10075F0002077AC3EA940F500302077A78FF79FFF2
:10076F007A0F02077A780079007AF0C3E524956151
:10077F00500AC374019524500B020798E54A20E7ED
:10078F000E020798E54A30E706884689478A4822CD
:10079F0078A5E6FAC3E54933F8E54A33F9D10EE90E
:1007AF0030E70BC3E89480E994FF4013E1D2C3E82C
:1007BF00947FE994005002E1D2787F7900E1D278FA
:1007CF008079FFE820E715C3E52398F84009C3E8CF
:1007DF00940140030207F978010207F9E8F42401B4
:1007EF002523F840030207F978FF884B2278A6E605
:1007FF00FAA847A94812060EE930E70CC3E894019E
:10080F00E994FF401602082EC3E894FFE9940050C4
:10081F000302082E78FF790002082E780179FFE98C
:10082F0020E715C3E54B98F84009C3E8940140034E
:10083F000208557801020855E8F42401254BF840C9
:10084F000302085578FF88242278FF20692879A1B0
:10085F00E76023E541601F74FF8541F0848539F01F
:0F086F00306A0375F005A4F8C5F0600278FFC386
:10087E00E895645002A864886322C3E5409440E57D
:10088E00419401E5635003140199046002F563225B
:10089E007883E6F520120F1A75E89012054675E872
:1008AE009030EDFDA8BDA9BE120FC0756E2C756FF0
:1008BE0000C3740013FD742C606613FC742C2CFCA6
:1008CE0074003DFDECFAEDFBC3E89AE99B4014E59C
:1008DE006E242CF56EE56F3400F56FEA2CFAEB3DC5
:1008EE00FB80E5AE6EAF6FC3E56F13F9E56E13F8DF
:1008FE00C3E913F9E813F87A03C3E913F9E813F817
:10090E00DAF7AA201A7009756E00756F0002092EAB
:10091E001AEA6008EE28FEEF39FFDAF88E6E8F6F56
:10092E002275E890227883E6FF30EDF9A8BDA9BEC6
:10093E000570C3E57094084052757000E9FA79A00D
:10094E00E76044EA7007E571601B020967C3E8952A
:10095E00716010E5715006600C140209730460F9A1
:10096E00020973E571F571C3946D401B7561C0C3C7
:10097E0094044013756180C39404400B756140C3A9
:10098E009404400375610075BB0622EFC3940160A9
:10099E001F742C601BC3E894FFE994035012C3E844
:1009AE00956EE9956F5009E561600C15610209C5F8
:1009BE00E561F460020561A861C3E524985002A8C0
:1009CE0024C3E89562400AA862E562F4600385627A
:1009DE006188258826E570B4070375BB1022743232
:1009EE0079A787F0A4C5F0A2F733F8C3E895614064
:1009FE0002A861882288248825882688642275406A
:100A0E00007541F022C2AF75C820A8CCA9CDAA3A74
:100A1E0030CF010A75C824D2AFAB3BAC3C883B89C2
:100A2E003CC3E89BF8E99C206908F9306602612214
:100A3E00417CAD3D8A3DF9EA9DFA600478FF79FF6D
:100A4E00AE3EAF3F8B3E8C3FA83BA93CC3E89EF821
:100A5E00E99FF9C3E54113FBE54013FAE82AF54097
:100A6E00E93BF54150067540FF7541FF41C9AA406B
:100A7E00AB41AC40AD417E047F02C3EB9404400D0C
:100A8E001E1FC3EB94084005206A021E1FC3ED1300
:100A9E00FDEC13FCDEF7C3EA9CFAEB9DFBEF60095D
:100AAE00C3E913F9E813F8DFF7EA28FAEB39FB8A02
:100ABE00408B4150067BFF8B408B41C3EB94025021
:100ACE0002D2663069047F0341F47892E6FFC3E5F3
:100ADE0037948240110FC3E53794A040010FC3EF46
:100AEE00940640027F057E02E541C4540FF9E541AC
:100AFE00C454F0F8E540C4540F28F8C3E89EFAE950
:100B0E009400FB4009C3EA9402EB940050047A026D
:100B1E00E4FB616EAA40AB41EBC4FEEAC4540F4E37
:100B2E00FCC3EA9CFAEB9400FBC3E813C313F8EA88
:100B3E0028FAEB3400FB8A408B41C3EB940240024F
:100B4E00C2667802EBC4FE7B00EAC4540F4EFAC3B1
:100B5E00EA98FA4005C3940250027A027892E6FFB0
:100B6E00306002616E855192855293D26043E68069
:100B7E00C3E49AF8E49BF930660261FAE8FAE9FBFD
:100B8E00D3E913FDE813FC88518952C3EF94036037
:100B9E0038EF20E00DE82CF8E93DF9ECFAEDFB0218
:100BAE000BC3E828F8E939F9C3E82402F8E9340060
:100BBE00F97AFE7BFFC3EF9403400E8A538B548861
:100BCE004D894E8C4F8D50812E885389548A4D8B72
:100BDE004E8C4F8D503069127553F07554FF754F12
:100BEE00F07550FF7551F07552FF812EE8FAD3E87B
:100BFE0013FC8851C3EF94036020EF20E007E82C2C
:100C0E00F8ECFA811AE8282402F87AFEC3EF94036E
:100C1E0040088A53884D8C4F812E88538A4D8C4FB5
:100C2E00E568C3335002646BF56830600281387535
:100C3E003402D26043E680E52D54066034A840A904
:100C4E0041C3E913F9E813F8C3E913F9E813F830CF
:100C5E006904E92440F9C2AF53E67F759100C3E4FD
:0F0C6E0098F594E499F595759104D26043E6806A
:100C7D00D2AF22D264754300752000306C0375200D
:100C8D0040020C9FD264754300752040306C037593
:100C9D00200078017901206620E52D54066002C2FE
:100CAD00647914E541C313700104F8C39414400230
:100CBD007814306904781B791B206010E543600CB3
:100CCD00306903D53404D26DA14A91400543E59BAB
:100CDD00F45440B52002A13430690908C3E89940A5
:100CED00011881C620640A08C3E8994002819F81DA
:100CFD00C6C264C2AF53E67F75910030661275941B
:100D0D00007595F8759104D26043E680D2AF819F4E
:100D1D00E5417EFFC3334005C3334001FEC3E49E6E
:100D2D00759400F595A111C3E53394015002819F8F
:100D3D00306402819FD802A14881C6C26DC2AF53F3
:100D4D00E67F759100855394855495759104854D75
:100D5D0092854E93D26043E680D2AFE52D54066066
:100D6D0008206A020533020D86306D0D206C0A20B5
:100D7D0064071581158102162622780030640278E9
:100D8D0001E53775F007A4F9E5F028F5F0E9A2F0D3
:100D9D0013A2F113A2F213F537C3947850037537EC
:100DAD0078C3E53795384008D265C292C290C2919A
:100DBD00306002A1BD854F92855093D26043E6808D
:100DCD0022207D16C2AF754202C294D295306202C6
:100DDD00D290D2AF759F11020FBDC2AF754202C244
:100DED0094D293306202D292D2AF759F11020FBD91
:100DFD00307243207D20C2AF75420390013A757B5E
:100E0D0010C290C293306204D291C11BD294D2AF62
:100E1D00759F01020FBDC2AF75420390013A757BFC
:100E2D0010C292C295306204D291C13BD294D2AF1E
:100E3D00759F21020FBD207D17C2AF754203900132
:100E4D0015C290306202D291D2AF759F01020FBDD3
:100E5D00C2AF754203900115C292306202D291D297
:100E6D00AF759F21020FBD207D16C2AF754204C222
:100E7D0095D293306202D291D2AF759F21020FBDF0
:100E8D00C2AF754204C293D295306202D291D2AFF5
:100E9D00759F01020FBD307243207D20C2AF754298
:100EAD0005900129757B20C291C294306204D292C3
:100EBD00C1C1D295D2AF759F11020FBDC2AF7542A0
:100ECD000590014B757B08C291C294306204D2909B
:100EDD00C1E1D293D2AF759F11020FBD207D17C214
:100EED00AF75420590010BC291306202D292D2AF22
:100EFD00759F11020FBDC2AF75420590011FC291C2
:100F0D003062EBD290D2AF759F11020FBD207D16CE
:100F1D00C2AF754206C293D294306202D292D2AF62
:100F2D00759F01020FBDC2AF754206C295D29430B6
:100F3D006202D290D2AF759F21020FBD3072432055
:100F4D007D20C2AF75420190014B757B08C292C2E4
:100F5D0095306204D290E167D293D2AF759F210292
:100F6D000FBDC2AF754201900129757B20C290C2A1
:100F7D0093306204D292E187D295D2AF759F010270
:100F8D000FBD207D17C2AF75420190011FC2923077
:100F9D006202D290D2AF759F21020FBDC2AF7542D2
:100FAD000190010BC290306202D292D2AF759F01B7
:100FBD00C26522900109757B00C292C290C291C296
:100FCD0095C293C294C2622278807607087607088C
:100FDD0076010876040876FF0876FF08760908760C
:100FED0002087601087601788C760108760008767D
:100FFD00B40876FF0876FF0876FF0876030876FFBB
:10100D000876010876FF0876250876D008767808E8
:10101D0076C80876040876FF08760108760008760B
:10102D007A08760A0876010876010876000876FFB8
:10103D00087600227887E6FFC272BF0302D272786B
:10104D0088C27DE630E102D27DC27E7889E630E14C
:10105D0002D27EC3EF94026008758E01D273021026
:0F106D0073758E00C273227880E6149000809312
:10107C0078A5F67881E6149000809378A6F67886A9
:10108C00E61490008D9378A7F6789FE6F8700575B6
:10109C006B0001BAC3E8941140027811E82828F5D6
:1010AC006B256B256B28F56C256B2828F56D7886E0
:1010BC00E6F539C394025003753902789CE675380D
:1010CC00FFB402037538A0B4030375388278A3E625
:1010DC001490009A93F566120FC022227896E6FAC5
:1010EC007897E6FB7888E6B40305C3EB940EFB30E7
:1010FC007F047A007BFFC3EB9AFCC3948250027C82
:10110C00827572000572EC8572F0A4C3E5F0947DD3
:10111C0040F222D27F11E81205551205557A007B58
:10112C00007C1012054BE55C2AFA74003BFBDCF3E7
:10113C007C04C3EB13FBEA13FADCF7FEC27F11E865
:10114C0022757C00757D00E5EF20E6037520000517
:10115C0020903FFFE520146006901DFF1460009363
:10116C0004600375EF1653D9BF7581C043FF80121D
:10117C00054675EF0643B203E5B3240220E70DF5EF
:10118C0021E5E320E0068521B343E301120FC0758E
:10119C0080FF75A40075F19175D47F75900075A5CD
:1011AC003F75F23F75D50075A60175E241120FC06F
:1011BC00E4F8F6D8FD756801120FD512167D7898F3
:1011CC008673753001C2AF12055F12056F1205559B
:1011DC0012057612055512057D1205551217A4122B
:1011EC00055F12055F12055AC2AF757C00757D0054
:1011FC0078FA79FA308707D9FBD8F7021C0011412D
:10120C00117411E711E878988673120FC075881065
:10121C0075890275C82475910475D84075A8227516
:10122C00B80275E690759B80759D0075D10E75BCE6
:10123C005875BB0675BA1175E880120546D2AF1207
:10124C00089E75360053DACF207E0343DA20307EB9
:10125C000343DA1043DA01C2D8C27112055FD261BE
:10126C007B037A0CE55B70077A0CDB030211F4123A
:10127C0005552070030211F4C270E55CC394024062
:10128C00E1E52F541F855E5DF55EB55DD5DAD5C2FF
:10129C006153DACF207E0343DA20307E0343DA1029
:1012AC00C2D8C27178A2E67008D274E52F54E0F56A
:1012BC002FC27575290012055A307409C3E529949B
:1012CC000A4002D27512054B78023074027800C3C2
:1012DC00E55C9840F0C2AF12056F12056F12056FF6
:1012EC00D2AF12055F754C0012054B788CE6C39497
:1012FC000150030213E1E530C3940150030213E1E2
:10130C00757CA5757DF1207435C3E55C94FF5003A5
:10131C000213E1C2AF120584D2AF12055AC3E55CC9
:10132C00940150EFC2AF12056F12055012056FD227
:10133C00AF12055AC3E55C94FF40E90218297F05FA
:10134C00D27F11E812055AC2AFC27F11E8AE5CC35E
:10135C00E55C947FD2AF500261F1120546C2AF1228
:10136C000584D2AFDFDA311FC3EE94057897F612FD
:10137C00055F1217AC7F0AD27F11E812055AC2AF73
:10138C00C27F11E8AE5CC3E55C947FD2AF50E6122D
:10139C000546C2AF12056F12055012056FD2AFDFB2
:1013AC00D6311FEE24037896F6F87997E7C394822A
:1013BC004003985006E824827897F612055F1216BF
:1013CC00BF1217DB12055A11E8C3E55C94FF5002FB
:1013DC00610C021829757C00757D00C3E55C954C89
:1013EC004003855C4C12055A78017988E7B40302F6
:1013FC007805C3E55C98400241F4C2AF1205841233
:10140C000584120584D2AF12055F753000E4F53106
:10141C00F5320531E531F4703F0532789AE67819EA
:10142C00146012783214600D787D14600878FA1408
:10143C006003753200C3E53298401D120FC01205CF
:10144C0046153275310078998673C2AF120584D275
:10145C00AF7898867312055A120550E52A7005303C
:0F146C00740221F478012074027806C3E55C98BD
:10147B0040A112055AE52A70030211F4C2AF120FF4
:10148B00C0E4F522F523F524F525F526F567D2AF53
:10149B007885E6C333F565E4F544F545F546F54740
:1014AB00F548F570F52CF52DF53775700875BB10F3
:1014BB0012054612092F30EDFDA8BDA9BEE970013A
:1014CB00F8887112093375700875BB101141C2AFE2
:1014DB007561FF1209EC852261852262852263D238
:1014EB00AF7522017524017525017526018560698B
:1014FB00756A017888E6B40307C27D307602D27D27
:10150B00D268D269753300120F1A120F49120A0CE6
:10151B00120A13120A0C120A13120A0C120C911251
:10152B000665120D87120DCE120A13120C80306E47
:10153B000312070520660312085830660312088849
:10154B00120D87120DFD120A13120C91306E03123D
:10155B000741120D87120E74120A13120C80306E93
:10156B000312079F120D87120EA3120A13120C916E
:10157B00306E031207FC120D87120F1A120A131288
:10158B00092F120C80120D87120F49120933120A00
:10159B001330692C856461856462856069756A01A5
:1015AB0079187A0CC3E533994009C269D26A8A3536
:1015BB000215CBC3E55C9401400302152702162EDE
:1015CB00306A1D206C1AE535147006C26AD26BA105
:1015DB0027F535C3E55C9401400302152702162E4F
:1015EB00753600C3E55F94014009856462856069C7
:1015FB00756A0178FA79A4E760027803C3E55F980E
:10160B005021307404E52A601A78F0306C0585643B
:10161B00617820C3E541985002A1270536E55C604F
:10162B0002C131753600C2AF120FC07887E6FE7665
:10163B000211417887EEF6E4F522F523F524F52522
:10164B00F526F565752C00752D00D2AF12055A12D3
:10165B000FC078A4E66006D292D291D29030740675
:10166B00E52A700221F4788DE6C39401400241D142
:10167B008119901A0D7820121701E520B4A50CA33F
:10168B00121701E520B45A0302169F120FD512163A
:10169B00BF0216BE901A0378807B0A121701A308AB
:1016AB00DBF9901A0F788C7B19121701A308DBF961
:1016BB00901A2822C2AF121744121721901A0074E5
:1016CB000E121706A37407121706A374151217062A
:1016DB00901A0378807B0A121705A308DBF9901A7E
:1016EB000F788C7B19121705A308DBF91217571209
:1016FB001735901A2822E493F622E6438F01538F75
:10170B00FDFFC3E583941C400122EF857CB7857DEB
:10171B00B7F0538FFE22438F02438F01857CB78531
:10172B007DB7901A0DF0538FFC22901A0D74A5F112
:10173B0006901A0E745AF106227A3079D0782090DE
:10174B001A40F101E520F709A3DAF7227A3079D0B4
:10175B00901A40E7F10609A3DAF922AB74A875BB1E
:10176B0001027980BB02027981BB03027982BB043F
:10177B00027994BB05027983BB06027986BB07020B
:10178B007992BB08027987BB0902799CBB0A027963
:10179B0088BB0B027989E8F7227C0512055FDCFB1D
:1017AB0022C2AF12056F12057612057D1205841247
:1017BB00055012056F12057612057D120584120570
:1017CB005012056F12057612057D120584D2AF22D9
:1017DB00C2AF12058412057D12057612056F120534
:1017EB005012058412057D12057612056F120550F5
:1017FB0012058412057D12057612056FD2AF22AE4B
:10180B0074AF75C2AF12056F12056F12056F12051B
:10181B0050DEF2120584120550DFF8D2AF221217F8
:10182B00AC1217A41217A4757401757501757600A7
:10183B00110A7C05AD5C12055FC3ED955C70F5C3B9
:10184B00E55C9401400AC3E55C94FF403702186CD9
:10185B001217661216BF1217ACC2AF75EF1612171E
:0E186B00A4DCD10576C3E5769403500280C25A
:101879001217A40575E5741490009F93F808C3E541
:101889007598500280A91217A41217A40574C3E50C
:1018990074940C50028095120FD51216BFC2AF7501
:0518A900EF161217A468
:0319FD0002114D87
:101A00000E071507070104FFFF09020101A55A018E
:101A100000B4FFFFFF03FF01FF25D078C804FF01DA
:091A200000FF0A010100FF00FFB4
:101A40002358503335415357232020202020202075
:101A500023424C48454C4923463333302320202031
:101A60002020202020202020202020202020202076
:101C0000C2AFC2D353D9BF7581C043B20343FF8073
:101C1000752438752503B1DC7529A5752AF175E29F
:101C20004043F18053A47F75D4FFD2877DFA7803B7
:101C300079E67C10752200752300901DE97B0675FE
:101C400024987525013087028145208708D8FBD963
:101C5000F9DCF781B7308708D8FBD9F9DCF781B711
:101C6000B19CE493A3C39A6004DDC381B7DBDBB10D
:101C70008E6002812E7B08E493FAA3B16FDBF87AC1
:101C800030B16F752200752300B18EEAFCEBFDC305
:101C9000ED94FE400EB18E8A278B28ED30E0048A49
:101CA000828B83B18E7AC270D8C3ED94FE601950D6
:101CB000CEBD002BEC600F7520007521FF7529004B
:101CC000752A000200008100A827A9280809D80465
:101CD000D90281DCB192EA89AAF281CE0D81A3C337
:101CE000ED94035053EDA2E092007AC5C3E58294CF
:101CF00000E583941C508A200010438F02438F011B
:101D00008529B7852AB7F0300029A827A92808090E
:101D1000438F01538FFDD804D902A133C3E58394C7
:101D20001C4003A3A11689AAE28529B7852AB7F02A
:101D3000A3A116538FFC817F7AC1BD030CE493A34A
:101D4000FAB153DCF8B14B817F8181AA22AB23B178
:101D50006FEBFAEA6222752608C3E52313F523E543
:101D60002213F52250066323A0632201D526EAB18F
:101D7000DCB1DC75260AEAF4200102D287300102C8
:101D8000C287B1DCC3134002C201D526EB22B19257
:101D9000EAFB208702A192308702A197752608AE40
:101DA00024AF25C3EF13FFEE13FEB1E0B1DCC3EAAD
:101DB000133087024480FA30E703632201C3E5232E
:101DC00013F523E52213F52250066323A0632201B5
:101DD000D526D9E52265236523F52222AE24AF2539
:101DE0000E0FDEFEDFFCD20122424C48656C6934E6
:071DF000373163F3300601F7
:00000001FF
